:1074000080E189BD82E189BD09B400FEFDCF089508
:10741000AA2069F08091E9008F931092E90097D437
:1074200083FF01C016D58F9187708093E90008957E
:107430008EEF0090E10008220092E1000895F20131
:10744000F999FECFF2BDE1BD0895F9DFF89A80B554
:1074500008C0F5DF1FBA80BD0FB6F894FA9AF99A02
:107460000FBE31962F010895E0E0F0E085919491F0
:10747000019608958BEA34D0109289008AEF8093A8
:10748000880082E080936F0083E080938100EBE6C8
:10749000F7E785913AD0E737E1F781E08093D700AD
:1074A0008AE482BF1092D8001092E2001092DA00B3
:1074B0001092E10080E808D019BCAA241092E000E4
:1074C0005CD489E04DD481E98093D8000895A3E687
:1074D000B1E090E81AD08D939A95E1F7089586E08F
:1074E00008D010C083E005D08F2F0FD08E2F0DD085
:1074F00080E05E9A729809C005D085E0FADF05D079
:1075000080FDFDCF729A5E9808958EBD8DB587FF80
:10751000FDCF8EB508958FE08221E9F7F3DFE3E632
:10752000F6E090EB5C98892FF0DF80E1EEDF5C9A6B
:107530008191EBDF83E68E278F77D1F79395983B88
:1075400089F70895E3E6F1E097FC36C094FC4DC05E
:1075500092FE089596849920D1F3F894C089D78536
:1075600020E030E080E090E4AFEFBFEF11968919A2
:107570009040E0F72D01BD4F8D0127FD13C0E0E0E5
:10758000F8E011928EE7819392E4E11791939AE5E6
:1075900008F092E4E334C9F781931082BFDFFE0163
:1075A0002196A0DF94DFF901F6D420583F4F040D57
:1075B000151D9A9411F71DC28301282D60906C014E
:1075C00070906B0143D019F48823C1F708953801F6
:1075D00088243CD0C9F580916A01821709F483019F
:1075E00060906E0170906D01F4CF80E1982E6090F4
:1075F0006E0170906D012AD059F48823B1F7089577
:107600009FEF95FC03C096FE089591E097FB890ECD
:10761000662477248301222719D0B1F48823A1F3AB
:1076200080916A0136F0881650F4821730F02130CC
:1076300003C0881520F4281710F48301282F6090C8
:107640006E0170906D01E8CF3801822EF3014ADFA0
:107650003EDFC3E6D1E0E4E6F7E70990859108163E
:1076600021F4EB36D1F7088080104CCFC9E031DF30
:10767000CA95E9F7D0E195FC1FC094FC38C096FC90
:1076800001C051C0C3E6D2E0E3E6F6E098E088E747
:107690008E0F00840192E817E1F7884F099001925C
:1076A000E817E1F7C858DF4F9A9589F734DFC85FCC
:1076B000D340C33E49F749C0C3E6D6E0EBE5FAE064
:1076C00098E08E2F885702900086E817E1F73896E9
:1076D0000A900292E817E1F73897C857D0409A9578
:1076E00081F719DFC850DC4FC33E41F72EC0A3EE2F
:1076F000B6E0E3E6F6E09AE0C6E00D9080818025F2
:10770000807F802582958193A336B90709F4B2E082
:10771000E336F90709F4F2E0E336FC0771F7FBDE24
:10772000DA9529F712C0A3EEB9E0E3E6FAE092E0B9
:107730000E90829180258F70802582958083E3361C
:10774000F907B1F7E8DEDA9571F78827089580E840
:1077500080BF8DEA8093640089E98093650085E0AD
:1077600083BF889541524455424F59D5F08D14A19D
:10777000C881CFD9F1AF000000FFFFCFCFFFFFFFDF
:10778000FFCFCFFFFF0000FE067E7E06FE46565668
:1077900016FE0656461EFE3F61E9E3FFE3EBE3FFFC
:0877A000E3EBE3FFE16B3F00A6
:1077A8001201100102000008412336000100000008
:1077B800000109023E0002010080320904000001B4
:1077C8000202010005240010010424020405240615
:1077D8000001070582030800FF09040100020A00EE
:1077E80000000705040210000107058302100001CC
:1078000011241FBE04B714BE88E18093600010925B
:1078100060008EEF9AE09EBF8DBF222433242101A9
:107820003101410180E88AC00F928F939F931F928C
:107830000FB60F9211244F936F938091DA0080FF5F
:1078400037C023C00F920FB68F939F93EF93FF9390
:1078500088278093850080938400E0E5F1E09281A1
:10786000907261F490818917980B908309F45D9A66
:1078700091818917980B918309F4289A239411F424
:107880008315381EFF91EF9154C08091D80080FF7E
:107890000FC08091DA008E7F8093DA008091D9004A
:1078A00080FF04C0ADDD81E0A82E02C019BCAA246F
:1078B0008091E10080FF0BC04DD280FF08C04DD207
:1078C0008091D800806200DE19BC85E0A82E8091EE
:1078D000E10084FF1AC03ED284FF17C091DD809181
:1078E000D8008F7DF1DD8FEEA4DD34D28F7E8160F4
:1078F00037D280915301882331F48091E30087FDD2
:1079000002C081E001C084E0A82E8091E10083FFE5
:107910000CC020D283FF09C087EF8BDD82E0A82E48
:107920001092530185DD19D228D26F914F910F909B
:107930001F909F918F910FBE0F90189580936100BB
:1079400010926100B1E0B5BF82E085BF81EF85B9DB
:1079500087EE84B984E08DB984E48EB910BA83EFE0
:1079600081BB80E68BB980EF8AB980E58CBDBDBD57
:10797000A0E0E8EAF7E705900D92A035E1F78C91D9
:107980001D92BB30E1F7893B11F4AADDE0CE5F9A8E
:1079900004C07C9B02C068DD61F56CDD789456DE26
:1079A00071F0ABE9B7E0E7E7F7E790E105900D92FA
:1079B0009A95E1F7A059BF4FE73AB9F7B0DD56D035
:1079C00027DD80915201807881F48FB18095807F8E
:1079D00066991C9B8460982E13DE89EB8825809322
:1079E000FF0A8110AFDD92FC02C0332042F73CDD7C
:1079F00031F3F89489EB74DD81E08093E00010921C
:107A00006F0010928100109285001092840081E036
:107A100085BF15BE2E9A2F9A2D9A5D9A289A0C949E
:107A2000000093D107C044D102C0AA2039F08FD101
:107A300082FFFBCF85FFF7CF8091F1000895082EDC
:107A400083E084D185FD07C079D102C0AA2069F006
:107A50007ED180FFFBCF0092F100809152018072B5
:107A600021F45D9884E68093500108956ED182FFE1
:107A700021C180915201807221F4289884E680937C
:107A80005101CFDF182F853431F422248EE7382EB0
:107A9000D6DC8DE0F8C0843511F4C3DFFACF8C3426
:107AA000C1F38035B1F3843711F480E0ECC0813448
:107AB00029F4B7DF582EB5DF482EEBCF833539F4E4
:107AC000E4E6F7E78591BBDFEB36E1F7DDC086350D
:107AD00021F482E3B4DF81E3D6C0863761F481E329
:107AE000669B8E5F1C9B8F5FAADF8FB1809582950E
:107AF0008F708F5BC8C08837A9F493DF80935201E1
:107B0000289A84FD28985D9A83FD5D982E9A81FDC0
:107B10002E982F9A82FD2F982D9A80FD2D9887FD03
:107B20008824B7CF8A3649F48FE9E3DCC3E0EDDC83
:107B300086DFCA95E1F7E6DCA7C0833731F487E832
:107B40007EDF85E97CDF8EE19EC0823631F489E5F7
:107B500076DF80E074DF80E896C0823419F08736E3
:107B600009F07DC033245DDFD82F5BDFC82F59DFDC
:107B7000082F8354843008F085C0063411F4440C77
:107B8000551CF20110926F001736B9F4033489F4D2
:107B900083E0A9DCBADC8EB51EBC51DF0DB42197A1
:107BA000D1F7B0DC08C0063411F4859101C04DDC7A
:107BB00046DF2197C2F72F014AC00334A9F4E1112F
:107BC00004C08DDC88ED8FDC97DC89DC82E08BDC07
:107BD00028DF0DB48EBDCA95D9F7319697DC8CDCC1
:107BE000DA9569F72F0131C00634F1F49F01F437BB
:107BF000D8F4E4D119C015DF063461F4C0FB46F0B7
:107C0000F43728F4182E81E087BFE89511243296C6
:107C1000082E0AC0043439F4DF01B370AD59B94FEE
:107C20008D93319601C015DC21972AF7043431F485
:107C30002F01F370FE2B49F472DC07C0063429F4DF
:107C40002F01F901F43708F4B7D18DE0F8DE0634DE
:107C500011F45694479482E080936F0015C08237E8
:107C6000E1E049F08634E0E031F08E34E3E019F0F1
:107C7000813531F4E2E0F0E089E087BF849103C010
:107C80008B3111F08FE3DBDE83E0CFDB57D095FF44
:107C900003C009C0AA2071F05AD080FFFBCF4ED09C
:107CA00002C0AA2039F053D080FFFBCF84E0BDDBB7
:107CB0008BE745C00895E4E5F1E067E090915B0152
:107CC00080915C01913231F0913AF1F58132E1F528
:107CD00060D183C0823281F48191805B8191844044
:107CE00099F580915D0180FD2FC0F89481E080932B
:107CF000E0001092FF0A84CD803231F54AD1AA20EB
:107D0000E9F08530D9F023D083FD18C082FFF7CF8A
:107D100004C092DE8193615031F09091F300809124
:107D2000F200892BB1F7C4DF611549F704C0AA201E
:107D300029F0853019F00BD080FFF9CF8EE79091B4
:107D4000E80089238093E800089584E06EDB809149
:107D5000E80008958091E2000895FCDF8E7F806145
:107D60008093E200089582E061EC09D083E061E84D
:107D700002D084E060E842E103C080E060E042E0DD
:107D800054DB81E007D01092ED006093EC0040934B
:107D9000ED0008959091EB00892B8093EB000895FE
:107DA00060E0923029F0913029F4E0E062E102C015
:107DB000E2E16EE3F1E0089580915B0188234CF4E9
:107DC00002C0AA20C1F3C3DF82FFFBCF71CFAA207C
:107DD00091F3BDDF80FFFBCFB1CF409161015091A6
:107DE00062014617510520F0462F611509F4A6DF00
:107DF00050E022C0AA2061F1853051F1A8DF83FD57
:107E000057CFA5DF82FD21C080FF16C03091F3005F
:107E10002091F20006C081918093F10041502F5FC4
:107E20003F4F411519F028303105A8F350E02830B4
:107E3000310509F451E082DF4115E1F65523D1F611
:107E400004C0AA2029F0853019F081DF82FFF9CF24
:107E50002FCFEBE5F1E0F0DD8193E336E1F72BDFA7
:107E600076DF83FF91C080915B0190915C0191303E
:107E700009F170F09330F1F0953009F444C0963078
:107E800009F456C0983009F460C0993059F767C0BA
:107E9000823841F780915F01C7DA2091EB001092A0
:107EA000E90077D02295269521702093F100109259
:107EB000F10052C0882311F08230A1F68F71823018
:107EC00089F680915D018823D1F420915F012770AC
:107ED00049F22093E9008091EB0080FF10C09330BD
:107EE00011F480E20BC080E155DF81E0880F2A9514
:107EF000E9F78093EA001092EA0088E04BDF1092E5
:107F0000E90047D02AC0882391F410915D011068E0
:107F10000FB7F8943ED050DF1ADF80FFFDCF1093EB
:107F2000E300103883E009F482E0A82E0FBF2CC0D4
:107F30008058823048F580915D0190915E0130DF7C
:107F4000603011F126D049DF1FC08038E9F421D01C
:107F5000809153018093F100F1DE2EDF15C088235C
:107F600099F490915D01923078F49093530111D07F
:107F700023DF80915301882321F48091E30091E075
:107F800087FD94E0A92EEFDEE2DE83FF089580E214
:107F900001DF87EFD4CEA3E6B1E0F437B8F40ED01A
:107FA00090E40D901D9081E087BFE89532969A95F8
:107FB000C1F71124E058F04085E001C083E001D012
:0E7FC00081E187BFE89507B600FCFDCF08956C
:067FFA003231CECFFBDCAA
:040000030000740085
:00000001FF
